:02000000D32803
:10000800FD28A601A500BA172730A4001030182033
:100018000330A400E8301820A40164301820A4019B
:100028000A30182025082328A3002608A20025083E
:10003800A100B2202108031DBA13BA1B0800303EE4
:10004800A7003E0884000930A80003103020A70C40
:10005800A80B2A28031430288413BA1D3F28000847
:100068003C043A1D3C068000841700083C04031C2D
:100078003C0680004A2800083C04031C3C063A1948
:100088003C06800084173C0980054A283A0D063949
:10009800A1005320A200A10A532000006D280030BF
:1000A8008A00210882070134993403343934003432
:1000B80060340C34FD34A401A300FF30A307031CF3
:1000C800A407031CCE280330A200E6306D20612867
:1000D800A201FC3EA100A209031C7828FF30000001
:1000E800A10703187328A1076400A20F722808004B
:1000F800A201A401A30002309728A201A401A30031
:1001080003309728A201A401A30001309728A20177
:10011800A401A30006309728A30004309728A20161
:10012800A401A3000530A90024082202031D9E286B
:10013800230821020430031801300319023029056D
:10014800031DFF30CE280038031DFF300405031DB2
:10015800FF30CE280404031DFF30CE28A601A501D8
:100168001030A700220DA50DA60D2308A50224080E
:10017800031C240FA6020318C8282308A50724086F
:100188000318240FA6070310A10DA20DA70BB6286C
:100198002108CE28831303138312640008004D102E
:1001A800CD10CA01D201D301D0010330D100C6015C
:1001B800C7011030C8002730C900831681133E30AC
:1001C80086008501831207309F0031309000C030CF
:1001D8008B00831601308C008312DC30C3000B3097
:1001E800C2000C30CB00CC01CF01C101C401C50154
:1001F8005829A000030E8301C0000A08BB00430869
:100208008E0042088F00C10A0C103B088A00400E7D
:100218008300A00E200E090064000A304102031C6E
:10022800572983168C0183124108A100A2010A30C4
:10023800A300A401B220B3002208B4003308CF07FA
:100248004108A100A2010A30A300A401B220B30012
:100258002208B4003308C40734080318013EC50750
:100268004108A100A2010A30A300A401B220250878
:10027800C100831601308C0064003C3083124F02A9
:10028800031C57293C30CF02CC0A64003C304C0296
:10029800031C5729CC01CB0A64000D304B02031C08
:1002A80057290130CB000800DC25102164005208D2
:1002B800013C031DAC294408A1004508A200A40183
:1002C80009309020031DAC290930C4020030031CFA
:1002D800013EC5026400CD1C92290630BE000130E3
:1002E800BC000630BA003930242020302420533096
:1002F800242065302420633024206F3024206E3081
:1003080024206430242020302420543024206930D4
:100318002420633024206B30242092250030861955
:100328000130A10000309320B300003006190130DD
:10033800A10000309320B500330884003508A720B9
:10034800B500B6006400350836040319AC290E243C
:1003580064005208003C031D872A5308A10000309E
:100368008120B3005308A10004308B20B500330866
:1003780084003508A720B500B600640035083604A7
:100388000319182A4408A1004508A200A40109304D
:100398009020031D182A0930C4020030031C013EB6
:1003A800C5026400CD1CFD290630BE000130BC002A
:1003B8000630BA003930242020302420733024201D
:1003C80065302420633024206F3024206E302420B0
:1003D80064302420203024207430242069302420E4
:1003E800633024206B30242020302420530805203B
:1003F8009225D30A003086190130A10000309320DD
:10040800B300003006190130A10000309320B50078
:10041800330884003508A720B500B6006400350805
:1004280036040319182AB2245308A1000530812084
:10043800B3005308A10007308B20B50033088400AF
:100448003508A720B500B60064003508360403193E
:10045800872A4408A1004508A200A4010A30902078
:10046800031D872A0A30C4020030031C013EC5025E
:100478006400CD1C662A0630BE000130BC00063080
:10048800BA0031302420303024202030242073302A
:10049800242065302420633024206F3024206E30DF
:1004A8002420643024202030242074302420693013
:1004B8002420633024206B3024202030242053084B
:1004C80005209225D30A640008305302031C6D2AC4
:1004D800D301003086190130A10000309320B30009
:1004E800003006190130A10000309320B500330810
:1004F80084003508A720B500B60064003508360426
:100508000319872AB2244E08A1004F089320B3008C
:10051800003086190130A10000309320B50033085F
:1005280084003508A720B500B60000300619013050
:10053800A10000309320B70035083604840037083E
:10054800A720B700B8006400370838040319B32A95
:100558006400CD1CB12AE6239D254F08CE0000304B
:1005680086190130A10000307C20B3000030061944
:100578000130A10000307C20B50033088400350824
:10058800A720B500B6006400350836040319DC2A34
:1005980005108316051083128510831685108312A3
:1005A800051183160511831285118316851183128F
:1005B800003086190130A10000307C20B3000030E3
:1005C80006190130A10000309320B50033088400DB
:1005D8003508A720B500B6006400350836040319AD
:1005E8000E2B46240930CF0764003C304F02031C11
:1005F8000E2B3C30CF02CC0A64003C304C02031C6A
:100608000E2BCC01CB0A64000D304B02031C0E2BC1
:100618000130CB00003006190130A10000307C20E9
:10062800B300003086190130A10000309320B500D6
:10063800330884003508A720B500B60064003508E3
:1006480036040319512B7C240930CF02640065302D
:100658004F02031C512B3C30CF07CC03640065309C
:100668004C02031C512B3B30CC00CB034B08A100A0
:1006780000307C20B3004B08A10064308620B50010
:10068800330884003508AE20B500B600640035088C
:1006980036040319512B0C30CB0000308619013079
:1006A800A10000309320B300003006190130A100EA
:1006B80000309320B500330884003508A720B50022
:1006C800B60064003508360403196B2B6C235929CE
:1006D8004608A1004708A2004908A400480883204A
:1006E800031DA12B64004A08003C031D802B051440
:1006F8008316051083129D2B64004A08013C031DD4
:100708008A2B85148316851083129D2B64004A0852
:10071800023C031D942B05158316051183129D2B8E
:1007280064004A08033C031D9D2B8515831685111B
:100738008312C60A0319C70AE52B64005108500240
:100748000318CE2B64004A08003C031DB02B051487
:10075800831605108312CD2B64004A08013C031D43
:10076800BA2B8514831685108312CD2B64004A0892
:10077800023C031DC42B0515831605118312CD2BCE
:1007880064004A08033C031DCD2B8515831685118B
:100798008312DE2B0510831605108312851083162D
:1007A800851083120511831605118312851183168E
:1007B80085118312D00A64000B305002031CE52B0C
:1007C800D001080064004A08003C031DF02B051402
:1007D8008316051083120D2C64004A08013C031D82
:1007E800FA2B85148316851083120D2C64004A0891
:1007F800023C031D042C05158316051183120D2CCC
:1008080064004A08033C031D0D2C851583168511C9
:1008180083120800051483160510831285158316A4
:100828008511643083125F2005108316051064302B
:1008380083125F20051583160511643083125F202B
:10084800851183168511643083125F208514831601
:100858008510643083125F200511831605116430FA
:1008680083125F20051483160510643083125F20FD
:10087800851083168510643083125F20CA01C60173
:10088800C701080005148316051083128515831601
:1008980085110A3083125F200510831605100A306F
:1008A80083125F200515831605110A3083125F2015
:1008B8008511831685110A3083125F2085148316EB
:1008C80085100A3083125F200511831605110A303E
:1008D80083125F200514831605100A3083125F20E7
:1008E8008510831685100A3083125F20CA0108001C
:1008F80005148316051083128514831685100A3093
:1009080083125F200510831605100A3083125F20BA
:100918000515831605110A3083125F20851083168A
:1009280085100A3083125F208515831685110A30D9
:1009380083125F200511831605110A3083125F2088
:100948000514831605100A3083125F20851183165B
:1009580085110A3083125F20CA01080064004A0822
:10096800003C031DCA2C0514831605108312851537
:1009780083168511643083125F20051083160510D5
:10098800643083125F200330CA001F2D64004A08B8
:10099800013C031DE12C8514831685108312051470
:1009A80083160510643083125F2085108316851026
:1009B800643083125F20CA011F2D64004A08023C7C
:1009C800031DF92C0515831605118312851483164A
:1009D8008510643083125F20051183160511643079
:1009E80083125F200130CA001F2D64004A08033CAF
:1009F800031D112D85158316851183120515831680
:100A08000511643083125F208511831685116430C7
:100A180083125F200230CA001F2D851583168511A9
:100A2800643083125F20051083160510643083122A
:100A38005F200330CA00C601C701080064004A08E5
:100A4800003C031D3A2D05148316051083128514E6
:100A580083168510643083125F20051083160510F5
:100A6800643083125F200130CA008F2D64004A0869
:100A7800013C031D522D851483168510831205151C
:100A880083160511643083125F2085108316851044
:100A9800643083125F200230CA008F2D64004A0838
:100AA800023C031D6A2D0515831605118312851551
:100AB80083168511643083125F2005118316051192
:100AC800643083125F200330CA008F2D64004A0807
:100AD800033C031D812D851583168511831205148A
:100AE80083160510643083125F20851183168511E3
:100AF800643083125F20CA018F2D851483168510F8
:100B0800643083125F200510831605106430831249
:100B18005F200130CA00C601C70108000630BE00C8
:100B28000130BC000630BA000A3024200D302420E1
:100B380008000630BE000130BC000630BA00433061
:100B4800242075302420723024207230242065300F
:100B580024206E3024207430242020302420743047
:100B68002420693024206D30242065302420203052
:100B780024206930242073302420203024204B087E
:100B880005203A3024204C0805202E3024204F0818
:100B980005202D302420410805200630BE000130F4
:100BA800BC000630BA000A3024200D30242008008A
:100BB8000514831605108312851083168510831279
:100BC8000511831605118312851183168511831269
:100BD8008617831686138312061783160613640076
:100BE8008312061EF92DD201FB2D0130D200922569
:100BF8000630BE000130BC000630BA004730242061
:100C080065302420613024207230242020302420B4
:100C1800433024206C3024206F302420633024207B
:100C28006B30242020302420493024206E302420AA
:100C38006930242074302420693024206130242035
:100C48006C302420693024207A3024206930242014
:100C58006E3024206730242092250630BE000130F3
:100C6800BC000630BA002830242063302420293004
:100C780024202030242032302420303024203030EA
:100C880024203930242020302420413024206C3086
:100C98002420613024206E30242027302420733013
:100CA800242020302420453024206C302420653036
:100CB80024206330242074302420723024206F30A4
:100CC80024206E30242069302420633024202030F2
:100CD800242050302420723024206F3024206A30A1
:100CE800242065302420633024207430242073307D
:100CF800242092250630BE000130BC000630BA0020
:100D08004430242065302420733024206930242086
:100D1800673024206E30242065302420643024205D
:100D280020302420623024207930242020302420D0
:100D3800413024206C302420613024206E3024205F
:100D48002030242050302420613024207230242088
:100D5800653024206B302420683024209225922589
:020D6800080081
:02400E00463F2B
:00000001FF
